:020000040000FA
:02000000AF2827
:08000800A100030EA0002E0868
:10001000B2002F08B300AB0B122800006820A52007
:100020001030AB00000000000B118B173208AE003F
:100030003308AF000B11200E8300A10E210E090022
:1000400082073F3406345B344F3466346D347D347C
:1000500007347F34673480340130A50089002208DA
:100060004620A50D2508890023084620A50D250852
:1000700089002408462008000530A700A7030319BB
:100080000800FF30A600A60B43283E2800002020D1
:1000900088003C2088018901080083160130850012
:1000A0000301880089008312850188018901080005
:1000B00083168E309F00831240309F000800831605
:1000C00087308100A0308B0083120130AB00080024
:1000D0001F140A30A800A80B6B281F151F196E28C3
:1000E00083161E088312A9001E08AA000800031028
:1000F0001030AC00B401B501B601AF0DAE0DB60DB8
:10010000B50DB40DAC0B85280034363084008F203B
:10011000353084008F20343084008F207D280330D8
:100120000007AD00AD19800030300007AD00AD1BF9
:100130008000003435080F39A2003608F039A300DA
:10014000A30E36080F39A4000800A90C0310AA0C4E
:100150000318A9172908AF002A08AE000800A0015B
:10016000A101A201A301A401A501A601A701850186
:10017000880189018316880186018701890185012B
:10018000831203134D2058205F20AA2077209A2045
:040190002C20C52832
:02400E00F93F78
:00000001FF
